:020000040800F2
:10000000D8060020191500080103000803030008A2
:10001000070300080B0300080F030008000000009E
:1000200000000000000000000000000013030008B2
:10003000150300080000000017030008190300085A
:100040003315000833150008331500083315000870
:100050003315000833150008331500083315000860
:100060003315000833150008331500083315000850
:100070003315000833150008331500083315000840
:100080003315000833150008331500083315000830
:100090003315000833150008331500083315000820
:1000A0003315000833150008331500083315000810
:1000B000C1110008E5080008A9110008331500085F
:1000C00033150008331500083315000833150008F0
:1000D000331500088D14000833150008FF040008CC
:1000E000331500083315000833150008DFF80CD06D
:1000F00003F06CF8004800478B020008D806002087
:1001000030B58FB06748007BA8B166488568446801
:10011000002C01DB204600E060420090002D01DB56
:10012000284600E0684203465E48427B5EA102A882
:1001300003F07CF814E05B4885684468002C01DB20
:10014000204600E060420090002D01DB284600E0E0
:10015000684203465348427B5CA102A803F066F85C
:10016000102302AA0021084600F0D9FD0FB030BDCF
:1001700010B50024002001F048F80446012C1CD0E2
:10018000022C0AD0032C02D0042C2ED122E04548A8
:10019000007BC0434349087328E04248406800F5AB
:1001A0007A70404948600846406841F658318842B4
:1001B00002DD08463B49486018E03A484068A0F52F
:1001C0007A703849486008464068002801DC002001
:1001D00048600BE03348407B18B90120314948732F
:1001E00002E000202F49487300E000BF00BF2D4807
:1001F000007B38B101203F49086000203E49C1F82A
:10020000B80106E000203B49086001203A49C1F8E6
:10021000B8012448407B68B1224840682149886081
:100220000846406870B90020324908603249C1F878
:10023000B80107E000201B4988602E4908602E495C
:10024000C1F8B8011748008941F65831081A2B49FE
:10025000088010BD10B501F03FF84FF4A06001F028
:10026000F1FE002141F61F4000F08AFE00F0BCFFC5
:1002700000F0E4FD00F079FC00200A49486001200C
:10028000487300201D49088010BDFFF7E3FF4FF4BD
:100290007A7001F05EF803E0FFF76AFFFFF730FFC6
:1002A000FAE70000980100202564202070776D5F38
:1002B00076616C3A25642C7461726765743A2564C2
:1002C00020202043572020202020200025642020AB
:1002D00070776D5F76616C3A25642C746172676526
:1002E000743A2564202020524556202020202020CA
:1002F00000000000B081214200802142402C0140DA
:10030000704700BFFEE700BFFEE700BFFEE700BF8B
:10031000FEE7704770477047704700000CB500203B
:10032000019000906C48006840F480306A49086091
:1003300000BF6948006800F4003000900198401C3C
:100340000190009818B90198B0F5A06FF1D16248FA
:10035000006800F4003010B10120009001E000209E
:1003600000900098012843D15C48006840F01000DC
:100370005A4908600846006820F0030008600846F3
:10038000006840F0020008605348406852494860E5
:100390000846406848600846406840F4806048600D
:1003A0000846406820F47C1048600846406840F4E5
:1003B000E81048600846006840F08070086000BFA0
:1003C0004548006800F000700028F9D042484068B5
:1003D00020F00300404948600846406840F00200B1
:1003E000486000BF3C48406800F00C000828F9D184
:1003F0000CBD10B5FFF792FF10BD10B53648006870
:1004000040F001003449086008464068344908401B
:100410003149486008460068324908402E49086062
:100420000846006820F4802008600846406820F4F0
:10043000FE0048604FF41F008860FFF7DAFF4FF0BE
:1004400000602949086010BD10B50021002000227D
:10045000214B5B6803F00C0121B1042906D0082967
:1004600028D107E0214B224C236027E01F4B204C72
:10047000236023E0184B5B6803F47010164B5B6835
:1004800003F48032022303EB904022B9194B43431B
:10049000174C23600DE0104B5B6803F4003323B16D
:1004A000144B4343124C236003E0104B4343104C66
:1004B000236003E00D4B0E4C236000BF00BF064BD2
:1004C0005B68C3F303130C4CE15C094B1B68CB4026
:1004D000074C236010BD00000010024000200240C5
:1004E0000000FFF8FFFFF6FE08ED00E000127A00C2
:1004F0000000002000093D0004000020704710B5F6
:1005000000246A4801F0DAFCC4B2694869490978F4
:10051000445468480078401C6649087008460078D2
:10052000642801DB0020087010BD002004E00021D9
:100530005F4A1154411C88B26428F8DB00215D4AEF
:100540001170704710B504460BE000BF40215748BA
:1005500001F01EFD0028F9D014F8011B534801F0EA
:10056000A9FC20780028F0D110BD10B50446FFF793
:10057000DCFF2046FFF7E6FF4FA0FFF7E3FF10BDCB
:1005800010B5044621464A4802F0D7FC08B10120C4
:1005900010BD0020FCE72DE9F04180460C461546D1
:1005A0001E4600270EE04046FFF7DFFFB0B200F026
:1005B000D0FE2046FFF7E4FF10B10120BDE8F08136
:1005C000781CC7B2AF42EEDB0020F7E710B564231A
:1005D00003223AA13AA0FFF7DEFF04464FF416705B
:1005E00000F0B7FE14B94FF0FF3010BD64230322B2
:1005F00032A135A0FFF7CFFF04464FF4167000F08C
:10060000A8FE14B96FF00100EFE7642303222BA1C9
:1006100031A0FFF7C0FF04464FF4167000F099FEBA
:1006200014B96FF00200E0E76423032223A132A093
:10063000FFF7B1FF04464FF4167000F08AFE14B9BC
:100640006FF00300D1E7642303221CA12EA0FFF763
:10065000A2FF04464FF4167000F07BFE14B96FF051
:100660000400C2E76423032214A12DA0FFF793FF27
:1006700004464FF4167000F06CFE14B96FF00500DC
:10068000B3E70020B1E710B504463223032228A1C6
:1006900028A0FFF780FFC82000F05BFE2046FFF790
:1006A00051FF642000F055FE10BD000000480040DE
:1006B000A8010020140000200D0000004F4B000096
:1006C00041540D0A0000000041542B43574D4F4444
:1006D000453D320D0A00000041542B435753415011
:1006E0003D225A48222C22313233343536373839BC
:1006F000222C352C330D0A0041542B4349504D55C3
:10070000583D310D0A00000041542B4349505345D8
:10071000525645523D312C353030300D0A00000024
:1007200041542B43495053544F3D300D0A000000B3
:100730003E00000041542B43495053454E443D3048
:100740002C31340D0A000000002807DA0121784A14
:1007500011600021774AC2F8B81106E00021744AFE
:1007600011600121734AC2F8B811011E01DB0A466B
:1007700000E04A42704B1A8070472DE9F04704466A
:100780006E4D6F4E002729466E48006802F0E7FB69
:100790006C49086031466B48006802F0E0FB804617
:1007A00041466848006802F064FC0746204602F0B3
:1007B0009EFC824664480168504602F022FC814655
:1007C000394602F024FC80465F480168404602F04A
:1007D000C6FB5D49086039464FF07E5002F011FCBF
:1007E000804658480168404602F011FC55490860AF
:1007F0005548006802F084FCBDE8F0872DE9F05F01
:1008000004460D46601B514908600968504A126849
:10081000881A02F06CFC83464E480168584602F084
:10082000F6FB80464948006802F061FC83464A486E
:100830000168584602F0EBFB8146414602F08FFB0F
:1008400007464648006802F052FC8246394602F0EC
:1008500086FB064602F054FC4049086008460068E2
:10086000B0F5E15F02DD4FF4E15008603B480068FD
:1008700010F5E15F02DA3A48384908603348006809
:100880003349086035480068BDE8F09F7FB50546EC
:100890000C460121022001F07AF9ADF80850ADF8BC
:1008A00004400020ADF80A00ADF8060001A92D486B
:1008B00001F00AFD012211462A4802F07CF81D20B1
:1008C0008DF8000003208DF801008DF80200012052
:1008D0008DF80300684601F0BAFB0121214802F0BF
:1008E0004FF87FBD10B5002401211E4802F011FB16
:1008F000E8B1022000F033FC1B4908600868FFF7EC
:100900003CFF194908600846407B30B10A465168EF
:100910001068FFF773FF044600E00024124884606B
:100920002046FFF711FF01210E4802F003FB10BD26
:10093000B081214200802142402C01400AD7A33CD3
:100940000000E0401C000020180000202C000020C7
:10095000280000202400002020000020300000207B
:10096000E0E3FFFF000400409801002010B54FF4C1
:100970000051F94800F0EFFE4FF40041F64800F056
:10098000EAFE4FF40041F44800F0E7FE4FF4005156
:10099000F14800F0E2FE10BD10B54FF40051EE48F2
:1009A00000F0D9FE4FF40041EB4800F0D6FE4FF4C2
:1009B0000041E94800F0CFFE10BD10B54FF40051E2
:1009C000E54800F0C8FE4FF40051E34800F0C5FED2
:1009D00010BD2DE9F04105462C464FF40051DE488C
:1009E00000F0BBFE00261CE0274607F08007802FA2
:1009F00004D13902D84800F0AEFE04E04FF40041C3
:100A0000D54800F0AAFE6006040E4FF40051D2480B
:100A100000F0A1FE4FF40051CF4800F09EFE701C84
:100A2000C6B2082EE0DBBDE8F08110B50446FFF742
:100A30009DFF7820FFF7CDFFFFF7BFFF0020FFF7F6
:100A4000C8FFFFF7BAFF2046FFF7C3FFFFF7B5FF68
:100A5000FFF7A2FF10BD10B50446FFF787FF78200F
:100A6000FFF7B7FFFFF7A9FF4020FFF7B2FFFFF73F
:100A7000A4FF2046FFF7ADFFFFF79FFFFFF78CFFB6
:100A800010BD70B504460D461DB1E0B2FFF7E3FF9F
:100A900002E0E0B2FFF7C9FF70BD70B50646002462
:100AA00018E004F1B0000021FFF7EBFF0021084639
:100AB000FFF7E7FF00211020FFF7E3FF002505E027
:100AC00001213046FFF7DDFF681CC5B2802DF7DB42
:100AD000601CC4B2082CE4DB70BD06E041F6650181
:100AE00000E0491E0029FCD1401E0028F6D17047C5
:100AF000014605E0002001E0421CD0B27B28FBDB70
:100B00000A1EA1F10101F5D1704770B504460D46EA
:100B100005F1B0000021FFF7B4FF102141EA1410E5
:100B20000021FFF7AEFF04F00F000021FFF7A9FF3F
:100B300070BD10B500218D20FFF7A3FF0021142008
:100B4000FFF79FFF0021AF20FFF79BFF10BD10B5FF
:100B500000218D20FFF795FF00211020FFF791FF66
:100B60000021AE20FFF78DFF10BD70B5002418E006
:100B700004F1B0000021FFF784FF00210846FFF7D1
:100B800080FF00211020FFF77CFF002505E00121F8
:100B90000020FFF776FF681CC5B2802DF7DB601CD4
:100BA000C4B2082CE4DB70BD70B5002418E004F179
:100BB000B0000021FFF765FF00210846FFF761FF45
:100BC00000211020FFF75DFF002505E00121084608
:100BD000FFF757FF681CC5B2802DF7DB601CC4B25D
:100BE000082CE4DB70BD2DE9F04707460E46904621
:100BF000994600250024A8F12000C5B27F2F02DD10
:100C00000027B01CC6B2B9F1100F24D131463846C6
:100C1000FFF77BFF002408E004EB05114F4A505C0E
:100C20000121FFF72EFF601CC4B2082CF4DB701CFE
:100C3000C1B23846FFF769FF002409E004EB051153
:100C40000831464A505C0121FFF71BFF601CC4B20B
:100C5000082CF3DB12E031463846FFF756FF00243C
:100C60000AE005EB45013E4A02EB4101085D012126
:100C7000FFF707FF601CC4B2062CF2DBBDE8F0876B
:100C800010B50246012000E050430B1EA1F1010403
:100C9000E1B2F9D110BD2DE9FF5F074691461E462E
:100CA0000E9D4FF0000A002435E0301B401EC1B2FB
:100CB0000A20FFF7E5FFB9FBF0F00A21B0FBF1F2E3
:100CC00001FB1208BAF1000F14D1701EA04211DD11
:100CD000B8F1000F0CD1AB4605EBDB71491001FBFD
:100CE0000471C8B22B4620220199FFF77CFF10E067
:100CF0004FF0010AAB4605EBDB71491001FB0471B3
:100D0000C8B208F13001CAB22B460199FFF76BFF58
:100D100000BF601CC4B2B442C7DBBDE8FF9F2DE931
:100D2000F04104460F461546984600260FE0AA5D9E
:100D3000434639462046FFF756FF04F10800C4B287
:100D4000782C02DD0024B81CC7B2701CC6B2A85DA6
:100D50000028ECD1BDE8F081000C0140FA35000814
:100D6000D23300082DE9F04180460E461546002793
:100D700031464046FFF7C9FE00240AE0744A02EB00
:100D80008511085D0121FFF77CFE781CC7B2601C4D
:100D9000C4B2102CF2DB701CC1B24046FFF7B5FEA6
:100DA00000240CE06900491C694A02EB4111085D0E
:100DB0000121FFF766FE781CC7B2601CC4B2102C7C
:100DC000F0DBBDE8F0812DE9F05F06460F46904666
:100DD0001C46DDF828A04FF0000BE11704EB517121
:100DE000C910A4EBC10131B92046E11704EB5171E0
:100DF000C1F3C70506E02046E11704EB5171C910A5
:100E0000491CCDB23D4615E029463046FFF77DFE30
:100E1000B1460BE059460BF1010B1AF80100012114
:100E2000FFF72FFE09F1010000F0FF09C145F1DBDA
:100E3000681CC5B2A542E7DBBDE8F09F08B50121FB
:100E4000082000F097FE4FF42040ADF8000010207D
:100E50008DF8030003208DF8020069463D4800F03C
:100E6000CDFB4FF420413B4800F075FC4FF4487037
:100E700000F06FFA0021AE20FFF703FE00210846C4
:100E8000FFF7FFFD00211020FFF7FBFD00214020B0
:100E9000FFF7F7FD0021B020FFF7F3FD00218120CF
:100EA000FFF7EFFD0021FF20FFF7EBFD0021A12060
:100EB000FFF7E7FD0021A620FFF7E3FD0021A820B2
:100EC000FFF7DFFD00213F20FFF7DBFD0021C820F9
:100ED000FFF7D7FD0021D320FFF7D3FD00210846FF
:100EE000FFF7CFFD0021D520FFF7CBFD00218020AB
:100EF000FFF7C7FD0021D820FFF7C3FD0021052023
:100F0000FFF7BFFD0021D920FFF7BBFD0021F12035
:100F1000FFF7B7FD0021DA20FFF7B3FD0021122013
:100F2000FFF7AFFD0021DB20FFF7ABFD00213020F4
:100F3000FFF7A7FD00218D20FFF7A3FD002114205E
:100F4000FFF79FFD0021AF20FFF79BFD08BD0000CC
:100F500034000020000C014008B50121082000F0F9
:100F600009FE4FF4A040ADF8000010208DF80300FA
:100F700003208DF8020069462A4800F03FFB08BDB7
:100F800030B589B005460C46FFF7E6FF0121C802DF
:100F900000F0F0FD0121042000F0ECFD4FF40060B2
:100FA000ADF8200018208DF8230003208DF82200D2
:100FB00008A91D4800F022FBADF81850ADF8144008
:100FC0000020ADF81A00ADF8160005A9174801F089
:100FD0007BF96020ADF804000120ADF80600002088
:100FE000ADF80A00ADF80C0001A9104801F0A9F90C
:100FF00001A90E4801F07FFA01210C4801F0CCFC58
:1010000008210A4801F0ECFD0821084801F007FE1C
:101010000121064801F0B4FD0121044801F0B0FCB3
:1010200009B030BD000C014000080140002C014017
:1010300000B587B00121084600F0A9FD0121042078
:1010400000F098FD0320ADF8000004208DF80300A7
:101050006946614800F0D2FA04A801F061FC002062
:10106000ADF810004FF6FF70ADF814000020ADF899
:101070001600ADF8120004A94FF0804001F024F9E9
:1010800000231A4603214FF0804001F02CFD01A8F7
:1010900001F059FC0A20ADF80C0001A9400701F04D
:1010A000A6FB0121880701F031FF012211469007BC
:1010B00001F081FC00214FF0804001F0F5FE01219C
:1010C000880701F05DFC07B000BD00B587B00121C5
:1010D000042000F05CFD0121082000F04BFDC02041
:1010E000ADF8000004208DF8030069463B4800F08D
:1010F00085FA04A801F014FC0020ADF810004FF6AA
:10110000FF70ADF814000020ADF81600ADF8120025
:1011100004A9334801F0D8F800231A4603213048C7
:1011200001F0E1FC01A801F00EFC0A20ADF80C0072
:1011300001A92B4801F05BFB0121294801F0E6FEE3
:1011400001221146264801F036FC0021244801F016
:10115000ABFE0121224801F013FC07B000BD01469F
:10116000022904D003290BD0042919D10FE04FF034
:101170008042928C10B200224FF080439A8411E09A
:10118000184A128810B20022164B1A800AE0144A3C
:101190002432128810B20022114B24331A8001E04D
:1011A000002000BF00BF70470D48103000880C4879
:1011B0001030008820F00100094910310880704784
:1011C0004FF08040008A4FF08040008A20F00100FC
:1011D0004FF080410882704700080140000C014038
:1011E000000800402404004008B50121182000F048
:1011F000C1FC48208DF803004EF20100ADF800005C
:101200006946334800F0FAF908BD10B5044614B138
:101210000120304908702F48007800283BD04FF457
:1012200000412B4800F07DFA80B14FF480412848FE
:1012300000F077FA50B14FF40051254800F071FAF0
:1012400020B10121224800F06CFA20BB0A2000F0F6
:1012500080F800201F4908704FF400411C4800F03E
:1012600060FA08B9012010BD4FF48041184800F021
:1012700058FA08B90220F6E70121154800F051FAA2
:1012800008B90320EFE74FF40051114800F049FA84
:10129000E0B90420E7E74FF400410D4800F041FABF
:1012A000012813D181030A4800F03BFA01280DD12F
:1012B0000121074800F035FA012807D1410304480D
:1012C00000F02FFA012801D1024908700020CAE776
:1012D000001001407401002010B56FF0040000F010
:1012E00000FF2E4800682E49B0FBF1F02D49087030
:1012F0000846007800EB4001C1EBC0104FF6FF71CB
:1013000001EAC0002849088010BD0146254A12782C
:101310004A434FF0E0235A6100229A611A4612694B
:1013200042F001021A6100BF4FF0E022106900F0A4
:1013300001021AB100F48032002AF5D04FF0E02209
:10134000126922F001024FF0E0231A6100229A6133
:1013500070470146144A12884A434FF0E0235A610D
:1013600000229A611A46126942F001021A6100BF16
:101370004FF0E022106900F001021AB100F480324F
:10138000002AF5D04FF0E022126922F001024FF05E
:10139000E0231A6100229A617047000000000020DB
:1013A00000127A007601002078010020014600BF7B
:1013B000704700BF544A128802F04002002AF9D058
:1013C000C2B2514B1B1D1A80704770B505460E46C0
:1013D000002400BF0BE000BF40214B4800F0D8FDC7
:1013E0000028F9D0295D484800F064FD641CB4422F
:1013F000F1DB70BD10B586B00446012144F2040053
:1014000000F0B8FB4FF40070ADF8140003208DF825
:10141000160018208DF8170005A93C4800F0EEF8DA
:101420004FF48060ADF8140004208DF8170005A972
:10143000364800F0E3F825208DF8000003208DF8F1
:1014400001008DF8020001208DF80300684600F0CD
:10145000FEFD01940020ADF80800ADF80A00ADF8DB
:101460000C00ADF810000C20ADF80E0001A92648C4
:1014700000F027FC012240F22551234800F0B9FC7E
:101480000121214800F0A9FC06B010BD10B540F2C2
:1014900025511D4800F092FD10B31B4800F00EFDD1
:1014A000C4B21B48008800F40040C8B9184800883E
:1014B00000F4804060B10A2C03D000201449088059
:1014C00020E01348008840F400401149088019E0EA
:1014D0000D2C06D10E48008840F480400C4908804D
:1014E00010E00B480088C0F30D000A490C5408486E
:1014F0000088401C0649088008460088C72801DD8E
:101500000020088010BD00000038014000080140A4
:10151000800100200C020020064880470648004752
:10152000FEE7FEE7FEE7FEE7FEE7FEE7FEE7FEE793
:10153000FEE7FEE7FB030008ED00000810B50446D7
:10154000CC48844208D10121042000F02DFB002169
:10155000042000F029FB46E0C748844208D101215D
:10156000082000F021FB0021082000F01DFB3AE0DC
:10157000C248844208D10121102000F015FB00214F
:10158000102000F011FB2EE0BD48844208D101215B
:10159000202000F009FB0021202000F005FB22E0C4
:1015A000B848844208D10121402000F0FDFA002112
:1015B000402000F0F9FA16E0B348844208D1012136
:1015C000802000F0F1FA0021802000F0EDFA0AE01E
:1015D000AE48844207D10121801500F0E5FA0021D0
:1015E000A01500F0E1FA10BD10B50121084600F089
:1015F000DBFA0021012000F0D7FA10BD2DE9F041FF
:10160000024600250026002000230024002791F830
:1016100003C00CF00F0591F803C00CF0100CBCF1E6
:10162000000F03D091F802C04CEA050591F800C004
:10163000BCF1000F31D0146800202BE04FF0010CFA
:101640000CFA00F3B1F800C00CEA03069E4220D168
:1016500083004FF00F0C0CFA03F7BC4305FA03FCB0
:101660004CEA040491F803C0BCF1280F06D14FF0F6
:10167000010C0CFA00FCC2F814C00AE091F803C097
:10168000BCF1480F05D14FF0010C0CFA00FCC2F878
:1016900010C0401C0828D1D31460B1F800C0BCF1C0
:1016A000FF0F34DD546800202EE000F1080C4FF0ED
:1016B000010808FA0CF3B1F800C00CEA03069E42D8
:1016C00021D183004FF00F0C0CFA03F7BC4305FA4D
:1016D00003FC4CEA040491F803C0BCF1280F05D1C7
:1016E00000F1080C08FA0CF8C2F8148091F803C055
:1016F000BCF1480F07D100F1080C4FF0010808FABF
:101700000CF8C2F81080401C0828CED35460BDE805
:10171000F0814FF6FF710180022181700421C170B8
:1017200070470246002093680B400BB1012000E097
:10173000002070470146886880B27047024600204A
:10174000D3680B400BB1012000E000207047014638
:10175000C86880B2704701617047416170470AB143
:10176000016100E041617047C16070474FF4803211
:101770000A4382618161826182698269704702469F
:101780000020434B18684FF68073184040EA02105F
:1017900008433F4B186070473E49C8617047F0B539
:1017A0000A46002300240021002500F00046B6F17F
:1017B000004F02D1364EF16901E0354E7168C0F339
:1017C000034583B200F44016B6F5401F08D121F05E
:1017D00070612F4E766826F070662D4F7E6012E0A5
:1017E00000F48016B6F5801F06D1032606FA05F42C
:1017F000A14341F0706106E0460D360103FA06F69A
:10180000B14341F0706122B1460D360103FA06F68C
:10181000314300F00046B6F1004F02D11C4EF16199
:1018200001E01B4E7160F0BD30B500228B071C0F2C
:101830000F2303FA04F2164B08338C1053F82430AC
:101840009343134C08348D1044F8253023468C10F4
:1018500053F824308C07240F00FA04F423430C4C73
:1018600008348D1044F8253030BD0A49DC31086059
:101870007047000000080140000C014000100140CA
:101880000014014000180140001C014000200140EC
:101890000000014000002042DF48006840F00100E5
:1018A000DD49086008464068DC490840DA4948607C
:1018B00008460068DA490840D749086008460068C9
:1018C00020F4802008600846406820F4FE0048604C
:1018D0004FF41F0088607047CF49096821F48031B8
:1018E000CD4A11601146096821F480211160B0F5DC
:1018F000803F03D0B0F5802F0ED106E0C6490968BD
:1019000041F48031C44A116007E0C349096841F4D9
:10191000A021C14A116000E000BF00BF704710B5B0
:1019200001460022002300204A11012A02D1BA4CAC
:10193000236806E0022A02D1B74C236A01E0B64CC4
:10194000636A01F01F02012494401C400CB1012085
:1019500000E0002010BD38B50020009000240025D4
:1019600000BF3120FFF7DBFF05460098401C0090C8
:101970000098B0F5A06F01D0002DF2D03120FFF714
:10198000CEFF08B1012400E00024204638BD014606
:101990000020A14A106820F0F80040EAC100106061
:1019A0007047A04908607047024600209A4B58686B
:1019B00020F47C1042EA01031843974B58607047AB
:1019C00098490866704701460020934A506820F005
:1019D00003000843506070478F48406800F00C00D7
:1019E0007047014600208C4A506820F0F000084300
:1019F0005060704701460020874A506820F4E0603C
:101A000008435060704701460020834A506820F424
:101A1000605040EAC1005060704729B17E4A527A56
:101A200002437D4B5A7204E07B4A527A82437A4BDE
:101A30005A7270477B49D8310860704701460020D0
:101A4000754A506820F440400843506070470021B8
:101A5000714A20321170704A82F82010012802D099
:101A600004280AD104E001216B4A2032117005E0FC
:101A70000521694A2032117000E000BF00BF7047A5
:101A80006949086070476449096A0143624A116202
:101A90007047654944390860704730B5002100221D
:101AA000002400235C4D6D6805F00C0121B1042970
:101AB00005D0082923D105E05C4D056022E05B4D8F
:101AC00005601FE0544D6D6805F47012524D6D684D
:101AD00005F48034022505EB92421CB9544D554360
:101AE00005600BE04C4D6D6805F400351DB1504D9F
:101AF0005543056002E04D4D5543056002E04B4DF6
:101B0000056000BF00BF444D6D6805F0F001090994
:101B1000484D6B5C0568DD4045603F4D6D6805F4E0
:101B2000E061090A434D6B5C4568DD4085603A4DD4
:101B30006D6805F46051C90A3E4D6B5C4568DD4037
:101B4000C560354D6D6805F44041890B3A4D6B5CBD
:101B5000C568B5FBF3F5056130BD29B12E4A526960
:101B600002432D4B5A6104E02B4A526982432A4BAF
:101B70005A61704729B1284A92690243264B9A61FB
:101B800004E0254A92698243234B9A61704729B148
:101B9000214AD2690243204BDA6104E01E4AD2692D
:101BA00082431D4BDA61704729B11B4AD268024358
:101BB000194BDA6004E0184AD2688243164BDA60A7
:101BC000704729B1144A12690243134B1A6104E0A9
:101BD000114A12698243104B1A6170471249403909
:101BE000086070470F49C86470470B49C871704757
:101BF0000948406A40F080700749486270470146D2
:101C00000020054A92680A400AB1012000E0002045
:101C10007047014988727047001002400000FFF8C9
:101C2000FFFFF6FE000042428004424200127A00AA
:101C300000093D00820100209201002010B50446F9
:101C4000FB48844209D101218803FFF7ADFF002141
:101C50004FF48040FFF7A8FF32E0F648844209D1F4
:101C600001214804FFF7ADFF00214FF40030FFF7DA
:101C7000A8FF25E0F048844209D101218804FFF73C
:101C8000A0FF00214FF48020FFF79BFF18E0EB48F6
:101C9000844209D10121C804FFF793FF00214FF4CA
:101CA0000020FFF78EFF0BE0E548844208D10121B8
:101CB0000805FFF786FF00214FF48010FFF781FF32
:101CC00010BD2DE9F04786B005460E460024A24619
:101CD00000BFA1460027B08900B100BF2F462C8A63
:101CE0004CF6FF700440F08804432C82AC894EF619
:101CF000F3100440B08831890843718908430443D4
:101D0000AC81AC8A4FF6FF400440B0890443AC82FA
:101D100001A8FFF7C2FEC648874202D1DDF810A035
:101D200001E0DDF80CA0A88900F4004040B10AEB06
:101D3000CA0000EB0A1031684900B0FBF1F807E077
:101D40000AEBCA0000EB0A1031688900B0FBF1F819
:101D50006420B8FBF0F004012009642101FB108924
:101D6000A88900F4004040B1322000EBC900B0FB6C
:101D7000F1F000F00700044308E0322000EB091006
:101D80006421B0FBF1F000F00F0004432C8106B099
:101D9000BDE8F0874FF41651016000218180C180B9
:101DA00001810C21418100218181704710B50246DB
:101DB0000020108A4FF2FF0318400B884C88234301
:101DC0008C882343CC8823431843108210BD002104
:101DD000018041808180C180704721B1828942F4B5
:101DE0000052828104E082894DF6FF731A4082819D
:101DF0007047F0B50346002400260025002040F679
:101E00006A17B94200D100BF1846C1F3421401F06D
:101E10001F06012707FA06F5012C01D10C3004E05A
:101E2000022C01D1103000E014301AB107682F43A2
:101E3000076002E00768AF430760F0BD1AB1838A0C
:101E40000B43838202E0838A8B4383827047028A3A
:101E50004FF6F0731A400282028A0A4302827047E8
:101E600082894FF2FF731A40828182890A438281FC
:101E7000704721B1828942F00202828104E08289A6
:101E80004FF6FD731A4082817047028A4FF6DF7366
:101E90001A400282028A0A430282704721B1028AF2
:101EA00042F48042028204E0028A4BF6FF731A4039
:101EB00002827047C1F30802828070470146888819
:101EC000C0F308007047818941F0010181817047AA
:101ED000028BD2B20283028B42EA01220283704754
:101EE000028B02F47F420283028B0A430283704713
:101EF00021B1828A42F02002828204E0828A4FF677
:101F0000DF731A408282704721B1828A42F0100248
:101F1000828204E0828A4FF6EF731A408282704711
:101F200021B1828A42F00802828204E0828A4FF65E
:101F3000F7731A408282704721B1828942F40042CD
:101F4000828103E08289C2F30E028281704721B14F
:101F5000828A42F40062828204E0828A4FF2FF7336
:101F60001A4082827047828A4FF6FB731A4082823F
:101F7000828A0A438282704721B1828A42F0020239
:101F8000828204E0828A4FF6FD731A408282704793
:101F900002460020B1F5007F00D100BF13880B403E
:101FA0000BB1012000E00020704701F40072B2F58F
:101FB000007F00D100BFCA430280704770B502465F
:101FC000002400230025002040F66A16B14200D10B
:101FD00000BFC1F3421501F01F03012606FA03F307
:101FE000012D02D19689334006E0022D02D1168AD6
:101FF000334001E0968A33400C12012606FA04F4BD
:102000001688344013B10CB1012000E0002070BDEF
:1020100010B50022002340F66A14A14200D100BF8F
:102020000A1201249440A3B2DC43048010BD0000D6
:10203000003801400044004000480040004C00408F
:102040000050004031490143314A1160704770B57A
:10205000002100230F22C47804B32D4C246804F41B
:10206000E064C4F5E064210AC1F10403CA40447885
:1020700004FA03F18478144021430901254C0678C1
:10208000A155047804F01F050124AC4005786D11BA
:10209000AD0005F1E025C5F8004109E0047804F041
:1020A0001F050124AC401C4D0678761145F82640EA
:1020B00070BD1A4A0A400243154B1B1F1A60704735
:1020C00039B1134A121D12680243114B1B1D1A60CD
:1020D00006E00F4A121D126882430D4B1B1D1A6049
:1020E0007047042808D14FF0E021096941F004014C
:1020F0004FF0E022116107E04FF0E021096921F083
:1021000004014FF0E0221161704700000000FA0561
:102110000CED00E000E400E080E100E080FFFF1F44
:1021200010B50446FE48844208D10121C014FFF7CF
:102130003BFD0021E014FFF737FDC4E0B4F1804F10
:1021400008D101210846FFF73CFD00210120FFF7DF
:1021500038FDB8E0F348844208D101210220FFF79E
:1021600030FD00210220FFF72CFDACE0EE48844258
:1021700008D101210420FFF724FD00210420FFF7EE
:1021800020FDA0E0E948844208D101210820FFF7A2
:1021900018FD00210820FFF714FD94E0E448844274
:1021A00008D101211020FFF70CFD00211020FFF7BE
:1021B00008FD88E0DF48844208D101212020FFF794
:1021C00000FD00212020FFF7FCFC7CE0DA4884427F
:1021D00008D101214014FFF7E7FC00216014FFF74C
:1021E000E3FC70E0D548844209D10121C804FFF71F
:1021F000DBFC00214FF40020FFF7D6FC63E0D04861
:10220000844209D101210805FFF7CEFC00214FF4DB
:102210008010FFF7C9FC56E0CA48844209D1012169
:102220004805FFF7C1FC00214FF40010FFF7BCFC8C
:1022300049E0C548844208D101214020FFF7C1FC94
:1022400000214020FFF7BDFC3DE0C048844208D19A
:1022500001218020FFF7B5FC00218020FFF7B1FCB1
:1022600031E0BB48844208D101218015FFF7A9FC69
:102270000021A015FFF7A5FC25E0B648844209D14E
:1022800001210804FFF790FC00214FF48030FFF794
:102290008BFC18E0B048844209D101214804FFF7C3
:1022A00083FC00214FF40030FFF77EFC0BE0AB48CD
:1022B000844208D101218804FFF776FC00214FF405
:1022C0008020FFF771FC10BD00220288944B9842D9
:1022D0000ED0994B98420BD0B0F1804F08D0914B63
:1022E000984205D0904B984202D0904B984204D12E
:1022F0004FF68F731A404B881A438D4B984207D084
:102300008C4B984204D04FF6FF431A40CB881A43B7
:1023100002808B8883850B880385814B98420BD084
:10232000854B984208D08B4B984205D08A4B9842F7
:1023300002D08A4B984201D10B7A03860123838213
:10234000704770B5002400220023058C4FF6FE76FE
:1023500035400584028C8388048B4FF68F752C40A2
:10236000B51E2C400D882C43751E2A400D892A432A
:102370004D882A436A4DA8420BD06F4DA84208D021
:10238000744DA84205D0744DA84202D0734DA842A6
:1023900013D14FF6F7752A404D892A434FF6FB7546
:1023A0002A408D882A434FF6FF652B404FF6FF5594
:1023B0002B408D892B43CD892B4383800483CD888B
:1023C0008586028470BD70B5002400220023058C30
:1023D0004FF6EF7635400584028C8388048B48F6EF
:1023E000FF752C404FF6FF452C400D884FF6FF76C9
:1023F00006EA05252C434FF6DF752A400D8906EACB
:1024000005152A434D8806EA05152A43444DA8427E
:1024100002D0494DA8421DD14FF67F752A404D8903
:102420004FF6FF7606EA05152A434FF6BF752A4098
:102430008D8806EA05152A434FF6FF352B404FF2EB
:10244000FF752B408D8906EA85052B43CD8906EA69
:1024500085052B4383800483CD880587028470BD66
:1024600070B5002400220023058C4FF6FF6635402E
:102470000584028C8388848B4FF68F752C404FF631
:10248000FC752C400D882C434FF6FF552A400D89D2
:102490004FF6FF7606EA05252A434D8806EA05250C
:1024A0002A431F4DA84202D0234DA8421DD14FF20E
:1024B000FF752A404D894FF6FF7606EA05252A4327
:1024C0004FF6FF352A408D8806EA05252A434EF649
:1024D000FF752B404DF6FF752B408D8906EA0515DB
:1024E0002B43CD8906EA05152B4383808483CD8851
:1024F0008587028470BD70B5002200230024058CFE
:102500004EF6FF7635400584038C8488828B48F62E
:10251000FF752A404FF6FF452A400D8820E0000055
:10252000002C01400004004000080040000C004066
:10253000001000400014004000340140004C0140F5
:10254000005001400054014000180040001C0040B1
:10255000002000400040014000440140004801408C
:102560004FF6FF7606EA05252A434DF6FF752B4008
:102570000D8906EA05352B434D8806EA05352B43C0
:10258000FA4DA84202D0FA4DA84208D14BF6FF7589
:102590002C408D894FF6FF7606EA85152C43848002
:1025A0008283CD88A0F84050038470BD828B4FF2A7
:1025B000FF331A408283828B4FF6FF7303EA0123B5
:1025C0001A4382837047F0B50C461546002200215D
:1025D0000026078C4EF6FF7C07EA0C070784828BE7
:1025E000018C4FF6FF7707EA043640F6FF473A4082
:1025F0004FF6FF7707EA05273A434FF6FF7707EADA
:1026000003373A43D94FB8420ED0D94FB8420BD016
:10261000B0F1804F08D0D74FB84205D0D64FB8425E
:1026200002D0D64FB84206D14DF6FF77394046F476
:102630008057394305E047F6FF57394044F4805747
:10264000394382830184F0BD828B4FF6F3731A40C5
:102650008283828B0A4382837047F0B50C4615460D
:10266000002200210026078C4FF6FF6C07EA0C07BA
:102670000784828B018C4FF6FF7707EA04264FF61A
:102680000C773A404FF6FF7707EA03172F433A4398
:10269000B64FB8420ED0B64FB8420BD0B0F1804F13
:1026A00008D0B44FB84205D0B34FB84202D0B34FB0
:1026B000B84206D14FF6FF57394046F48077394388
:1026C00005E04FF2FF57394044F480773943828365
:1026D0000184F0BD028B4FF2FF331A400283028B5C
:1026E0004FF6FF7303EA01231A4302837047F0B5E4
:1026F0000C461546002200210026078C4FF6EF7C81
:1027000007EA0C070784028B018C4FF6FF7707EA74
:10271000041640F6FF473A404FF6FF7707EA0337C3
:102720003A434FF6FF7707EA05273A438F4FB842FF
:102730000ED08F4FB8420BD0B0F1804F08D08D4FE4
:10274000B84205D08C4FB84202D08C4FB84206D167
:102750004FF6DF77394046F01007394305E04FF672
:102760005F77394044F01007394302830184F0BD9C
:10277000028B4FF6F3731A400283028B0A430283E3
:102780007047F0B50C46154600220021068C4FF626
:10279000FE773E400684028B018C4FF60C76324069
:1027A0007E1C06EA03162E433243704EB0420ED012
:1027B0006F4EB0420BD0B0F1804F08D06D4EB0429A
:1027C00005D06D4EB04202D06C4EB04206D14FF6ED
:1027D000FD76314044F00106314305E04FF6F576D1
:1027E000314044F00106314302830184F0BD70B5ED
:1027F00005460C465D4885420ED05D4885420BD0AB
:10280000B5F1804F08D05B48854205D05A488542D3
:1028100002D05A48854200D100E000BF208850B95C
:102820002389A28861882846FFF7ABFFE188284604
:10283000FFF79EFF25E0208804280AD12389A2887B
:1028400061882846FFF753FFE1882846FFF742FFDB
:1028500017E0208808280AD12389A28861882846A1
:10286000FFF7FBFEE1882846FFF7EEFE09E023892B
:10287000A28861882846FFF7A6FEE1882846FFF770
:1028800095FE70BD2DE9F04105460C460026012756
:10289000608808B9022600E00026A088012801D13E
:1028A000022700E001272088A0B92389A288618837
:1028B0002846FFF766FFE1882846FFF759FF23897E
:1028C0003A4631462846FFF712FFE1882846FFF7CF
:1028D00001FF13E02389A28861882846FFF707FFDC
:1028E000E1882846FFF7F6FE23893A463146284616
:1028F000FFF747FFE1882846FFF73AFFBDE8F08180
:102900000A884B881A438B881A43CB881A430B8951
:102910001A434B891A438B891A43A0F84420704705
:102920004FF6FF71818000210180C18041800172DA
:1029300070470021018041808180C18001814181F7
:102940008181C18170470021018041800121818006
:102950000021C18001817047002101804180818078
:10296000C18001814181818170470000002C0140BC
:10297000003401400004004000080040000C00400A
:1029800021B1028842F00102028004E002884FF681
:10299000FE731A400280704731B1B0F8442042F40F
:1029A0000042A0F8442005E0B0F84420C2F30E0233
:1029B000A0F8442070471AB183890B43838102E059
:1029C00083898B43838170478182704741EA020388
:1029D000A0F8483070471AB183890B43838102E025
:1029E00083898B438381704701894FF6F8721140C8
:1029F000018170470A46002101894FF68F73194003
:102A000011430181704730B504460D4629462046E2
:102A1000FFF7F0FF208940F00700208130BD2DE94D
:102A2000F04104460D4616461F46602D06D13B4632
:102A3000012231462046FFF75AFE05E03B460122BF
:102A400031462046FFF79DFE29462046FFF7D2FF7C
:102A5000208940F007002081BDE8F08130B50C46A8
:102A600000210189C9B24FF6FF7505EA0325154318
:102A700025432943018130BD2DE9F04105460E462D
:102A800017469846002443463A4631462846FFF703
:102A9000E5FF2C894FF6F870044044F007044FF628
:102AA0008F70044044F070042C81BDE8F081F0B5D3
:102AB00004460D4616461F463B46324629462046EA
:102AC000FFF7CCFF208940F480402081F0BD0185D4
:102AD000828270470A46002101884FF68F731940A1
:102AE000114301807047F0B50C4615461E46002183
:102AF000002200230189028B038C4FF6F8773940BE
:102B000021434FF6FC473A4040F201173A434FF653
:102B1000DD773B404FF6FF7707EA06172F433B432D
:102B2000018102830384F0BD0A460021018B4FF628
:102B30008F7319401143018370470A460021018BAE
:102B400048F6FF7319404FF6FF7303EA0223194357
:102B5000018370470A460021818B4FF68F7319401D
:102B60001143818370470A460021818B48F6FF7329
:102B700019404FF6FF7303EA02231943818370471C
:102B800021B1028842F08002028004E002884FF600
:102B90007F731A400280704721B1828842F004029C
:102BA000828004E082884FF6FB731A40828070476F
:102BB00021B1828842F00802828004E082884FF6C8
:102BC000F7731A408280704721B1828842F0010277
:102BD000828004E082884FF6FE731A40828070473C
:102BE0000A460021018B4FF6F77319401143018308
:102BF00070470A460021018B4FF2FF7319404FF6D0
:102C0000FF7303EA02231943018370470A46002138
:102C1000818B4FF6F77319401143818370470A4641
:102C20000021818B4FF2FF7319404FF6FF7303EAC7
:102C300002231943818370470A460021018B4FF616
:102C4000FB7319401143018370470A460021018B31
:102C50004FF6FF3319404FF6FF7303EA022319437F
:102C6000018370470A460021818B4FF6FB731940A0
:102C70001143818370470A460021818B4FF6FF3351
:102C800019404FF6FF7303EA02231943818370470B
:102C90000A460021018B4FF67F73194011430183CF
:102CA00070470A460021018BC1F30E014FF6FF73F6
:102CB00003EA02231943018370470A460021818BEE
:102CC0004FF67F7319401143818370470A460021F4
:102CD000818BC1F30E014FF6FF7303EA0223194300
:102CE000818370470A460021018C4FF6FD7319401D
:102CF0001143018470470A460021018C4FF6F77397
:102D000019401143018470470A460021018C4FF697
:102D1000DF7319404FF6FF7303EA0213194301846E
:102D200070470A460021018C4FF67F7319404FF619
:102D3000FF7303EA02131943018470470A46002116
:102D4000018C4FF6FF5319404FF6FF7303EA02233D
:102D50001943018470470A460021018C4FF2FF732A
:102D600019404FF6FF7303EA0223194301847047A9
:102D70000A460021018C4DF6FF7319404FF6FF7390
:102D800003EA023319430184704730B5002301245C
:102D90008C40A3B2048C9C430484048C02FA01F599
:102DA000ADB22C43048430BD30B5002304248C40E4
:102DB000A3B2048C9C430484048C02FA01F5ADB2E6
:102DC0002C43048430BD70B503460020002418460F
:102DD000183001258D40ACB21D8CA5431D8409B16E
:102DE000082909D100EB6100056825F07005056030
:102DF0000568154305600EE00D1FC5F34E05284418
:102E0000056825F4E045056005684FF6FF7606EA9B
:102E100002263543056070BD21B1028842F00202EE
:102E2000028004E002884FF6FD731A40028070476A
:102E300021B1028842F00402028004E002884FF6C9
:102E4000FB731A400280704721B1828842F08002F1
:102E5000828004E082884FF67F731A408280704738
:102E600002884FF6F7731A40028002880A430280F4
:102E7000704782884FF68F731A40828082880A4397
:102E80008280704702894FF6F8731A4002810289E6
:102E90000A430281704702894FF67F731A4002810C
:102EA00002890A4302817047818470478185704797
:102EB000818670470187704781877047A0F840106E
:102EC000704702884FF6FF431A40028002880A4387
:102ED000028070470146888E70470146088F704710
:102EE0000146888F70470146B1F84000704701469F
:102EF000888C70470146088D704702460020138A6F
:102F00000B400BB1012000E000207047CA43028251
:102F1000704730B50246002000230024158A05EAD8
:102F20000103958905EA010413B10CB1012000E009
:102F3000002030BDCA430282704730B505462A469C
:102F40000B4612F8010B13F8014B08B1A042F8D060
:102F50001CB1002802D06D1CF1E7284630BDF0B44A
:102F600080EA0102D40F4200B2EB410F02D20246C6
:102F7000084611464A0042D0C30DDDB2C1F3C75224
:102F8000AD1A202D35DAC1F3160141F4000204B167
:102F90005242C5F1200602FA06F12A411044B3EB71
:102FA000D05F23D0C4B1012DA0EBC35009DCF0BC2D
:102FB0004FF0004202EAC352DBB200F5000000F01D
:102FC000D7B8400000F1807000EBC350A0F18070D2
:102FD00040EAD170490009E0490841EAC071A0EB1C
:102FE000C35000F50000400800EBC350F0BC00F0F7
:102FF000B6B86142012202EB4101001BF6E7F0BCCA
:10300000704781F00041AAE780F00040A7E780EA1E
:10301000010210B502F00043400022D04A001FD048
:10302000010E01EB1261C0F35600C2F3560240F4E8
:10303000000042F40002A0FB022000047F391404C7
:1030400000D0401C50EA124001D44000491EC2B2D8
:103050000C0604EBD010401C4008802A02D003E08C
:10306000002010BD20F00100002900DA00201843E4
:1030700010BD30B480EA010202F0004530F0004299
:1030800021F0004013D090B1C30DD40DC2F316014E
:10309000C0F31600E41A41F4000140F400027D344C
:1030A000914201D3641C00E04900002C02DA30BCDC
:1030B000002070474FF400000023914201D3891A89
:1030C000034340084FEA4101F7D151B1914202D187
:1030D0004FF0004105E002D24FF0010101E06FF036
:1030E000010103EBC450284430BC00F038B8C10FD4
:1030F00080EAE0700844CA079623002100F038B83F
:1031000000F0004220F00040C10DC0F3160040F472
:1031100000007F2901DA00207047962903DCC1F105
:103120009601C84001E096398840002AF4D0404218
:10313000704730B50B46014600202022012409E0EB
:1031400021FA02F59D4205D303FA02F5491B04FA60
:1031500002F52844151EA2F10102F1DC30BD002960
:10316000A8BF7047401C490008BF20F0010070470D
:1031700010B4B0FA80FC00FA0CF050EA010404BF6D
:1031800010BC704749B1CCF1200421FA04F411FAC3
:103190000CF118BF012121430843A3EB0C01CB1D07
:1031A0004FEA00614FEA102042BF002010BC704778
:1031B00000EBC35010440029A4BF10BC7047401C52
:1031C000490008BF20F0010010BC7047064C074DB5
:1031D00006E0E06840F0010394E8070098471034E7
:1031E000AC42F6D3FCF786FFEC3B00080C3C000831
:1031F00030B58C1810F8012B12F00F0301D110F824
:10320000013B120906D110F8012B03E010F8015B15
:1032100001F8015B5B1EF9D101E001F8013B521E90
:10322000FBD1A142E6D3002030BD00000FB4084B13
:1032300010B504A902AA039800F01CF8044602A9DC
:10324000002000F0C1F8204610BC5DF814FB00001F
:10325000C933000802E008C8121F08C1002AFAD1C9
:1032600070477047002001E001C1121F002AFBD106
:10327000704700002DE9FF4F89B09B4604460025AA
:1032800006E025280BD05A460B999047641C6D1C0C
:1032900020780028F5D10DB02846BDE8F08F002732
:1032A000B8460122474900E0074314F8013F203B9C
:1032B00002FA03F00842F7D120782E2819D114F829
:1032C000010F47F004072A280ED06FF02F02207854
:1032D000A0F1300109290CD808EB880102EB41016B
:1032E00000EB0108641CF2E70A98641C50F8048B98
:1032F0000A9020780028CED0642808D0692806D00B
:1033000075281ED05A460B9990476D1C58E00A99B3
:103310004FF00A0901C90A91002802DA40422D2122
:1033200002E0390504D52B218DF82010012103E09E
:10333000F90704D02021F7E78A4608AE0DE0002106
:10334000FAE70A994FF00A0901C90A91F7E74946D5
:10335000FFF7EFFE303106F8011D0028F7D1ADEB85
:10336000060000F12009780701D44FF00108C84594
:1033700002DDA8EB090000E000208046002706E0FF
:1033800008A85A46C05D0B9990476D1C7F1C574595
:10339000F6DB04E030205A460B9990476D1CB8F1DB
:1033A0000001A8F10108F5DC05E016F8010B5A460A
:1033B0000B9990476D1CB9F10001A9F10109F4DCEA
:1033C000641C65E7092801000A68531C0B60107033
:1033D00070470000000000000000002F0000000007
:1033E0000700070000147F147F1400242A7F2A128C
:1033F000006264081323003649552250000005037B
:10340000000000001C224100000041221C000014AA
:10341000083E08140008083E0808000000A06000EC
:10342000000808080808000060600000002010087C
:103430000402003E5149453E0000427F40000042E8
:1034400061514946002141454B31001814127F104B
:10345000002745454539003C4A494930000171097A
:10346000050300364949493600064949291E00002E
:1034700036360000000056360000000814224100D5
:103480000014141414140000412214080002015105
:10349000090600324959513E007C1211127C007F0E
:1034A00049494936003E41414122007F4141221CA9
:1034B000007F49494941007F09090901003E41490E
:1034C000497A007F0808087F0000417F4100002002
:1034D00040413F01007F08142241007F40404040AE
:1034E000007F020C027F007F0408107F003E4141F4
:1034F000413E007F09090906003E4151215E007FDF
:10350000091929460046494949310001017F010155
:10351000003F4040403F001F2040201F003F4038F8
:10352000403F006314081463000708700807006137
:103530005149454300007F41410000552A552A5515
:10354000000041417F0000040201020400404040AD
:103550004040000001020400002054545478007FD1
:103560004844443800384444442000384444487FA8
:1035700000385454541800087E0901020018A4A40D
:10358000A47C007F080404780000447D40000040D3
:1035900080847D00007F102844000000417F4000AF
:1035A000007C04180478007C080404780038444443
:1035B000443800FC242424180018242418FC007C1F
:1035C0000804040800485454542000043F44402098
:1035D000003C4040207C001C2040201C003C40302F
:1035E000403C004428102844001CA0A0A07C0044BB
:1035F00064544C441414141414140000000000000B
:1036000000000000000000000000000000F80000C2
:103610000000000000333000000000100C06100C09
:103620000600000000000000000040C07840C078A4
:103630004000043F04043F040400007088FC08308C
:103640000000001820FF211E0000F008F000E01824
:10365000000000211C031E211E0000F008887000DD
:1036600000001E2123241927211010160E0000002F
:1036700000000000000000000000000000E018044E
:103680000200000000071820400000020418E000BB
:1036900000000040201807000000404080F08040FB
:1036A00040000202010F01020200000000F00000D1
:1036B00000000101011F01010100000000000000E5
:1036C000000080B07000000000000000000000005A
:1036D00000000001010101010101000000000000E3
:1036E000000000303000000000000000000080609A
:1036F0001804006018060100000000E0100808101F
:10370000E000000F102020100F00001010F8000043
:1037100000000020203F20200000007008080888DA
:1037200070000030282422213000003008888848AA
:1037300030000018202020110E000000C02010F8DA
:10374000000000070424243F240000F808888808AB
:1037500008000019212020110E0000E010888818B0
:103760000000000F112020110E0000380808C83892
:1037700008000000003F0000000000708808088872
:103780007000001C222121221C0000E010080810FB
:10379000E0000000312222110F00000000C0C00034
:1037A0000000000000303000000000000080000039
:1037B0000000000080600000000000008040201039
:1037C0000800000102040810200040404040404032
:1037D0004000040404040404040000081020408095
:1037E00000000020100804020100007048080808CA
:1037F000F0000000003036010000C030C828E8109A
:10380000E0000718272423140B000000C038E00054
:103810000000203C23020227382008F8888888709E
:103820000000203F202020110E00C03008080808AA
:103830003800071820202010080008F80808081091
:10384000E000203F202020100F0008F88888E808BA
:103850001000203F20202320180008F88888E8085E
:103860001000203F200003000000C0300808083886
:10387000000007182020221E020008F80800000897
:10388000F808203F210101213F20000808F808081E
:1038900000000020203F2020000000000808F80859
:1038A0000800C08080807F00000008F888C02818C9
:1038B0000800203F20012638200008F808000000FA
:1038C0000000203F20202020300008F8F800F8F801
:1038D0000800203F003F003F200008F830C00008EB
:1038E000F808203F200007183F00E01008080810E3
:1038F000E0000F10202020100F0008F8080808082A
:10390000F000203F210101010000E010080808102C
:10391000E0000F18242438504F0008F88888888861
:103920007000203F2000030C302000708808080839
:1039300038000038202121221C00180808F8080847
:1039400018000000203F2000000008F808000008D0
:10395000F808001F202020201F000878880000C8D9
:103960003808000007380E010000F80800F80008C9
:10397000F800033C0700073C0300081868808068D3
:10398000180820302C03032C30200838C800C83811
:1039900008000000203F2000000010080808C83878
:1039A00008002038262120201800000000FE020216
:1039B00002000000007F40404000000C30C00000CA
:1039C0000000000000010638C00000020202FE00F4
:1039D0000000004040407F0000000000040202029E
:1039E00004000000000000000000000000000000D3
:1039F00000008080808080808080000202040000BF
:103A000000000000000000000000000080808080B6
:103A100000000019242222223F2008F800808000A4
:103A20000000003F112020110E0000000080808067
:103A30000000000E1120202011000000008080886E
:103A4000F800000E112020103F20000080808080B0
:103A50000000001F222222221300008080F08888AC
:103A600088180020203F20200000000080808080F7
:103A70008000006B94949493600008F8008080802C
:103A80000000203F210000203F2000809898000087
:103A900000000020203F20200000000000809898B7
:103AA000000000C08080807F000008F80000808057
:103AB0008000203F24022D302000000808F800007C
:103AC00000000020203F2020000080808080808037
:103AD0008000203F20003F20003F808000808080C9
:103AE0000000203F210000203F20000080808080D7
:103AF0000000001F202020201F0080800080800008
:103B0000000080FFA12020110E00000000808080B6
:103B10008000000E112020A0FF8080808000808027
:103B2000800020203F212000010000008080808054
:103B300080000033242424241900008080E0808049
:103B400000000000001F2020000080800000008096
:103B50008000001F202020103F20808080000080F7
:103B6000808000010E300806010080800080008007
:103B700080800F300C030C300F00008080008080AC
:103B800080000020312E0E312000808080000080D7
:103B9000808080818E701806010000808080808087
:103BA00080000021302C2221300000000000807CA9
:103BB000020200000000003F404000000000FF0043
:103BC000000000000000FF0000000002027C8000F6
:103BD00000000040403F000000000006010102021A
:103BE0000404000000000000000000000C3C00087D
:103BF0000000002098010000F0310008D83C0008C7
:103C00009801002040050000643200089500A24A97
:103C100004B90102030406070809DB20416666F6C1
:103C200040CDCC8C3F001012101010FF109008886F
:103C30008888FF888888080010130444827F0180E8
:103C40008040432C10284681800E1310101010D095
:103C500030FF30D0121C101036100804020132FF61
:103C6000061401020408100D13FE222222FE00FE9B
:103C7000828292A29E2880601F0242827F0814FFE7
:103C8000402F102C43800B1590884C57A42454547B
:103C90008C8400101301018042221A0702428242E2
:103CA0003E0101010E1504E4242CB4252624B42C75
:103CB00024E4040C14FF02011E1212121E41827F22
:103CC0000212013011010203040102030406070875
:083CD0000902040608000000CF
:04000005080000ED02
:00000001FF
